:20FFD600E000E000E000E000E000E000E000E000E000E000E000E000E000FD00E000E000EE
:0AFFF600E000E000E000E000E000A1
:20C00000464C094B5420202020005350454349414C50524F472E3F20202000535045432E07
:20C0200050524F47204B4C41523F200050524F4752414D46454C00000000000000414E475A
:20C0400045204B4F443A00000000000000007300204E31202020204E32202020204E332030
:20C0600000492F4F20544553543F00494E47084E4720414B542E3A00555447084E47204189
:20C080004B542E3A0046454C484953544F52494B3F2020202000414E542E50524F472E3AE5
:20C0A000000050554D505449443A0000000044524946545241444552494E47202121205488
:20C0C000454D502031204F46465345543A0054454D502032204F46465345543A0073656B20
:20C0E000006D003F002E0050524F4752414D4D4552494E4720202000202000DF4320006D3D
:20C10000696E00204D4544202000205554414E200050002000300025006800094E4452413F
:20C12000204B4F443A0000000000000042525954205354520A4D4D454E000000004D415256
:20C140004B45524120494E53502E3F20200053540A545449443A000000000000000000563F
:20C1600009524D455220534B0A4C4A54414E4B004752414E554C4154004449534B415220B8
:20C18000202000534B0A4C4A4552202000564944415245203D2053544152542020004645B9
:20C1A0004C20485556520A52454C53452020005354094E4720485556454E20460A5220003C
:20C1C000202020202020202020202020202020200056415454454E46594C4C4E494E47200A
:20C1E000200046594C4C45522056415454454E2020200044524946544B4C415220202020DC
:20C200002020200046454C2046594C4C4E494E47202020200050524F562050524F475241B2
:20C220004D202020200046454C204859445241554C494B202020002020202053544F505017
:20C24000414420202020200046454C204B4C094D534B5944442020200046454C2053094B58
:20C260004552482E4E495608200046454C204B4F5247445249564E494E470046454C2053C7
:20C28000094B4252595441524520200046454C204D4F544F52534B59444420200046454CD3
:20C2A000200A482D534B594444202020200046454C2056415454454E545259434B20005317
:20C2C000544152543D4A412C203F3D4E454A20004C41444441205354414E444152443F2070
:20C2E000004C41444441205354414E444152443F3F00414E54414C2050524F4752414D3A17
:20C30000000000204449534B544944202000000000000000094E445241200A5652494741E0
:20C320002020200000534B0A4C4A54454D503A000000000000004449534B54454D503A0054
:20C340000000000000000053455041524154494F4E3A000000000000534B0A4C4A5449448E
:20C360003A00000000000000004E495608204449534B3A000000000000004E4956082053A1
:20C380004B0A4C4A3A000000000000464C094B54205449443A00000000000000534B0A4C0F
:20C3A0004A4D4544454C000000000000004B4C4152200A56524947412020202020005052BD
:20C3C0004F4752414D4D2E204B4C41523F2000454E474C4953483F2020202020202020007A
:20C3E000444555545343483F2020202020202020004652414E434149533F202020202020A8
:20C4000020005356454E534B413F20202020202020200053554F4D493F20202020202020F6
:20C42000202020004E454445524C414E44533F2020202020004954414C49414E4F3F20200D
:20C440002020202020004E4F52534B3F2020202020202020202000455350414E4F4C3F20BF
:19C46000202020202020200044414E534B3F2020202020202020202000F3
:20C4800046414E202020202020005350454349414C2050524F472E3F202000535045432EA8
:20C4A0002050524F472E204F4B3F200050524F4752414D204552524F5200000000494E5034
:20C4C000555420434F44453A0000000000007300204E31202020204E32202020204E33200B
:20C4E00000492F4F20544553543F00494E47084E4720414B542E3A00555447084E47204105
:20C500004B542E3A004552524F52204D455353414745532020004E4F2E50524F473A000095
:20C52000000050554D5054494D453A00000044524946545241444552494E472021212054B5
:20C54000454D502031204F46465345543A0054454D502032204F46465345543A00736563A3
:20C56000006D003F002E0050524F4752414D4D494E47202020202000202000DF4320006D0F
:20C58000696E002057495448200020572F4F202000500020003000250068004348414E4785
:20C5A0004520434F44453A00000000005455524E204D414348494E45204F4646004D415288
:20C5C0004B20494E5350454354494F4E3F00494D50554C53452D54494D453A0000000048B8
:20C5E000454154494E4720424F494C45522020004752414E554C455300574153484553201A
:20C6000020200052494E53455320202000434F4E54494E5545203D2053544152540045529F
:20C62000524F5220484F4F444D4F56454D2E00434C4F534520484F4F4420464F5220200004
:20C64000202020202020202020202020202020200057415445522D46494C4C494E472020E5
:20C66000200046494C4C53205741544552202020202000524541445920544F205741534852
:20C68000202020004552524F522046494C4C494E4720202000545249414C2050524F475205
:20C6A000414D4D4520004552524F52204859445241554C494353002020494E54455252552F
:20C6C00050544544202020004552524F5220484F4F44534146455459004552524F52205330
:20C6E000414645204C4556454C004552524F52205241434B204452495645004552524F52E7
:20C700002053414645545953572E20004552524F52204D4F544F5250524F542000455252AC
:20C720004F522053555045524850524F54004552524F52205741544552505245535300530F
:20C74000544152543D5945532020203F3D4E4F004C4F4144204445462E56414C5545533FAB
:20C76000004C4F4144204445462E56414C5545533F004E4F2E204F462050524F4752533AB6
:20C78000000000205741534854494D4520000000000000004348414E4745204F54482E56C2
:20C7A000414C3F200052494E53452D54454D503A000000000000574153482D54454D503A9F
:20C7C0000000000000000053455041524154494F4E3A00000000000052494E53452D5449DE
:20C7E0004D453A0000000000004C4556454C20574153483A0000000000004C4556454C20D0
:20C80000424F494C45523A0000000046414E54494D453A00000000000000000052494E53A7
:20C82000452D4147454E5400000000000046494E4953484544204F54482E56414C0050520F
:20C840004F47522E2046494E49534845442000454E474C4953483F202020202020202000EF
:20C86000444555545343483F2020202020202020004652414E434149533F20202020202023
:20C8800020005356454E534B413F20202020202020200053554F4D493F2020202020202072
:20C8A000202020004E454445524C414E44533F2020202020004954414C49414E4F3F202089
:20C8C0002020202020004E4F52534B3F2020202020202020202000455350414E4F4C3F203B
:19C8E000202020202020200044414E534B3F20202020202020202020006F
:20C900004C0E46544552202020005350455A49414C2050524F472E3F2020005350455A2E9F
:20C9200050524F472E204F4B3F20200050524F4752414D4D204645484C45520000434F4447
:20C94000452045494E474542454E3A0000007300204E31202020204E32202020204E3320C8
:20C9600000492F4F20544553543F00494E47084E4720414B542E3A00555447084E47204180
:20C980004B542E3A004645484C45524D454C44554E47454E2000414E5A2E50524F472E3A64
:20C9A000000050554D504544415545523A0044524946545241444552494E472021212054AA
:20C9C000454D502031204F46465345543A0054454D502032204F46465345543A0053656B37
:20C9E000006D003F002E0050524F4752414D4D494552554E47202000202000DF4320004D1F
:20CA0000696E00204D4954202000204F484E452000500020003000250068004E45554552DF
:20CA200020434F44453A0000000000005354524F4D2041425354454C4C454E0000494E5348
:20CA4000502E204D41524B4945522E3F2000494D50554C5344415545523A000000000048D3
:20CA60004549545A5420424F494C4552202020004752414E554C41540053500E4C454E20DB
:20CA80002020004B4C415253500E4C2000574549544552203D205354415254202000464569
:20CAA000484C2E4841554245424557472E20004841554245205343484C49455353454E0066
:20CAC0002020202020202020202020202020202000460E5220574153534552460E4C4C458A
:20CAE0004E00460E4C4C54205741535345522020202000424554524945425342455245497C
:20CB0000542020004645484C455220460E4C4C454E20202000564552535543482050524F9B
:20CB20004752414D4D004645484C2E4859445241554C494B2020002050524F4752414D4DC2
:20CB400053544F50502020004645484C2E4B4C454D4D53434855545A004645484C2E534972
:20CB600043482E4E4956454155004648454C2E4B4F5242414E5452494542004645484C2E67
:20CB8000534943482E534348414C54004645484C2E204D4F544F525343482E200046454884
:20CBA0004C200E482D53434855545A2020004645484C2E574153534552445255434B005377
:20CBC000544152543D4A4120203F3D4E45494E005745524B5357455254204C4144454E3FDB
:20CBE000005745524B5357455254204C4144454E3F00414E5A2E2050524F4752414D4D3ACE
:20CC00000000002053500E4C5A4549542000000000000000414E442E574552544520094E9C
:20CC200044524E3F004B4C415253500E4C544D503A000000000053500E4C54454D503A0012
:20CC40000000000000000041425452454E4E44415545523A000000004B4C415253500E4CF8
:20CC6000444155523A000000004E49562E2053500E4C454E3A00000000004E49562E2042CC
:20CC80004F494C45523A00000000004C0E4654455244415545523A00000000004B4C41527F
:20CCA00053502E4D49544C000000000000414E44455245205745525445204F4B3F0050527C
:20CCC0004F4752414D2E204645525449473F00454E474C4953483F20202020202020200047
:20CCE000444555545343483F2020202020202020004652414E434149533F2020202020209F
:20CD000020005356454E534B413F20202020202020200053554F4D493F20202020202020ED
:20CD2000202020004E454445524C414E44533F2020202020004954414C49414E4F3F202004
:20CD40002020202020004E4F52534B3F2020202020202020202000455350414E4F4C3F20B6
:19CD6000202020202020200044414E534B3F2020202020202020202000EA
:20CD800056454E54494C4552200050524F472E205350454349414C453F200050524F472E79
:20CDA00020535045432E204F4B3F200050524F4752414D4D452045525245555200494E5358
:20CDC0004552455220434F44453A000000007300204E31202020204E32202020204E33207D
:20CDE00000492F4F20544553543F00494E47084E4720414B542E3A00555447084E472041FC
:20CE00004B542E3A00414646495343482E2045525245555220004E425245205047522E3A3C
:20CE200000004455520B4520504D503A000044524946545241444552494E472021212054D5
:20CE4000454D502031204F46465345543A0054454D502032204F46465345543A007365639A
:20CE6000006D003F002E0050524F4752414D4D4154494F4E20202000202000DF4320006DA9
:20CE8000696E00204156454320002053414E532000500020003000250068004E4F5556452D
:20CEA000415520434F44453A00000000455441494E445245204D4143482E000000504F49CC
:20CEC0004E54204420494E53504543542E0054454D505320494D50554C533A000000004DDE
:20CEE000495345200D2054454D5020424F552E004752414E554C4553004C415645202020B1
:20CF000020200052494E43452020202000434F4E54494E5545203D205354415254004552D9
:20CF2000522E4645524D2E4341504F542020004645524D2E204341504F5420504F5552000D
:20CF4000202020202020202020202020202020200052454D504C495353414745204541559A
:20CF6000200052454D504C49542045415520202020200050520C5445204155204C41564198
:20CF8000474520004552524555522052454D504C4953532E005047522E204558504552494F
:20CFA0004D454E5420004552522E204859445241554C495155450020202020204152520C08
:20CFC00054202020202020004552522E4341504F5420534543555220004552522E4E4956E9
:20CFE000454155205345435552004552522E454E54522E50414E49455220004552522E49F7
:20D000004E54455252205345435552004552522E5345435552204D4F544555520045525265
:20D020002E20534555522053555243482E004552522E20505245535320454155202000533E
:20D04000544152543D4F554920203F3D4E4F4E0056414C2E4445462E205553494E453F20B3
:20D060000056414C2E4445462E205553494E453F3F004E4252452044452050524F47522ED8
:20D080003A0000204455522E4C41562E20000000000000004348414E4745204155545220CA
:20D0A00056414C3F00544D502052494E0F4147453A000000000054454D50204C415641477D
:20D0C000453A00000000004455522E20534550415241543A000000004455522E2052494E2C
:20D0E0000F4147453A000000004E49562E204C41564147453A00000000004E49562E204278
:20D100004F55494C4C3A00000000004455522E56454E54494C2E3A00000000004147454EE2
:20D12000542052494E0F2E00000000000050520C54204155545245533F20202020005052FE
:20D140004F47522E5445524D494E0B453F2000454E474C4953483F202020202020202000F2
:20D16000444555545343483F2020202020202020004652414E434149533F2020202020201A
:20D1800020005356454E534B413F20202020202020200053554F4D493F2020202020202069
:20D1A000202020004E454445524C414E44533F2020202020004954414C49414E4F3F202080
:20D1C0002020202020004E4F52534B3F2020202020202020202000455350414E4F4C3F2032
:19D1E000202020202020200044414E534B3F202020202020202020200066
:20D20000505548414C4C494E20004552494B4F49534F484A2E3F20202020004F484A454C3B
:20D220004D4F494E5449204F4B3F20004F484A454C4D4156495248452000000000414E4E8A
:20D2400041204B4F4F44493A0000000000007300204E31202020204E32202020204E33208A
:20D2600000492F4F20544553543F00494E47084E4720414B542E3A00555447084E47204177
:20D280004B542E3A0056494B41484953544F52494120202020004F484A454C2E4C4B4D3ABB
:20D2A000000050554D50505541494B3A000044524946545241444552494E472021212054DD
:20D2C000454D502031204F46465345543A0054454D502032204F46465345543A0073656B0E
:20D2E000006D003F002E004F484A454C4D4F494E5449202020202000202000DF4320004DA3
:20D30000494E00202B2020202000202D202020200050002000300025006800564149484445
:20D3200041204B4F4F44493A000000004B41544B414953452056495254410000004B495203
:20D340004A41205441524B49535455533F004B09594E4E4953545953494B413A00000048DD
:20D36000555548542E564544454E204C094D4D0052414550455355200050455355202020E6
:20D380002020004855554854454C5520004A41544B41203D20535441525420202000564944
:20D3A000524845204B5556554E4C494B45200053554C4A45204B55505520202020202000E8
:20D3C0002020202020202020202020202020202000564544454E54095954540A20202020F3
:20D3E000200054095954090920564554540920202020004B095954540A56414C4D495320BA
:20D400002020200056090952092054095954540A20202020004B4F454F484A454C4D4120E2
:20D420002020202020005649524845204859445241554C2E2020005649524845205059538D
:20D4400009595445545459005649524845204B5556554E52414A4120005649524845205469
:20D460005552564152414A412000564952484520504553554B4F5249202000564952484562
:20D480002054555256414B59544B2E005649524845204D4F4F54544F52492020005649521D
:20D4A000484520594C494B55554D2E202000564952484520564553495041494E452000536C
:20D4C000544152543D202B2020203F3D202D20004C415441412056414B494F3F2020202084
:20D4E000004C415441412056414B494F3F3F202020004F484A454C4D49454E204C4B4D3A78
:20D50000000000502D41494B413A000000000000000000004D55555441204D555554203FE8
:20D52000202020200048555548542E4C094D503A000000000000504553554C094D500A54F6
:20D540003A00000000000052454B45455420504F49533A000000000048555548542E4149F6
:20D560004B413A000000000000414E5455524920504553553A0000000000414E54555249A8
:20D580002048555548543A00000000505548414C4C2E41494B413A00000000004855554825
:20D5A000542E41494E453A0000000000004D5555542056414C4D49533F20202020004F4805
:20D5C0004A454C4D412056414C4D49533F2000454E474C4953483F2020202020202020004E
:20D5E000444555545343483F2020202020202020004652414E434149533F20202020202096
:20D6000020005356454E534B413F20202020202020200053554F4D493F20202020202020E4
:20D62000202020004E454445524C414E44533F2020202020004954414C49414E4F3F2020FB
:20D640002020202020004E4F52534B3F2020202020202020202000455350414E4F4C3F20AD
:19D66000202020202020200044414E534B3F2020202020202020202000E1
:20D6800056454E54494C41542000535045432E50524F472E5354414E443F00535045432E32
:20D6A0002050524F472E204F4B3F200050524F4752414D4D4120464F5554000000574143EC
:20D6C0004854574F4F52443A0000000000007300204E31202020204E32202020204E3320B6
:20D6E00000492F4F20544553543F00494E47084E4720414B542E3A00555447084E472041F3
:20D700004B542E3A00464F5554204D454C44494E47454E20200041414E542E50524F473A0D
:20D720000000504F4D5054494A443A00000044524946545241444552494E472021212054AD
:20D74000454D502031204F46465345543A0054454D502032204F46465345543A0073656391
:20D76000006D003F002E0050524F4752414D4D4552454E2020202000202000DF4320004DF1
:20D78000494E00204D4554202000204745454E2000500020003000250068004E4945555798
:20D7A0002E5741434854573A00000000484F4F4644534348414B2E2055495400004E415A30
:20D7C000494348542050554E543F20202000494D504F4C532054494A443A0000000000566C
:20D7E0004552572E20424F494C455220202020004B4F5252454C53200057415353454E207D
:20D800002020004E4153504F454C202000564552444552203D205354415254202000464FCE
:20D82000555420484F4544534C554954202000534C55495420484F4544202020202020009D
:20D840002020202020202020202020202020202000564F4F522056554C4C454E202020200C
:20D86000200056554C54205741544552202020202020004B4C415220562E20574153534569
:20D880004E202000464F55542056554C202020202020202000544553542050524F4752417A
:20D8A0004D4D41202000464F5554204F4C49455359535445454D0050524F47522E4F4E4403
:20D8C000455242524F4B2E00464F5554204B4E454C42455645494C2000464F555420574100
:20D8E0005445524E495645415500464F5554204B4F5246414E44522E202000464F555420F4
:20D9000044455552534348414B202000504F4D50204F56455242454C415354200044524FD5
:20D920004F474B4F4F4B20424556202020004C4147452057415445524452554B202000533B
:20D94000544152543D4A412020203F3D4E454500464142522E494E5354454C4C2E3F2020FF
:20D9600000464142522E494E5354454C4C2E3F3F200041414E542E50524F4752414D2E3AA5
:20D980000000002057415354494A443A2000000000000000414E44455245204745472E57D0
:20D9A000494A5A3F004E4153504F4C54454D503A00000000000057415354454D503A0000A3
:20D9C000000000000000004E412057415353454E3A000000000000004E4153504F4C544923
:20D9E0004A443A0000000000004E49562E2057415354414E4B3A000000004E49562E204254
:20DA00004F494C45523A000000000056454E542E2054494A443A0000000000004E4153502F
:20DA20004F454C4D49442E000000000000414E44455245204745472E204F4B3F2000505273
:20DA40004F4752414D2E4B4C4141523F202000454E474C4953483F202020202020202000EF
:20DA6000444555545343483F2020202020202020004652414E434149533F20202020202011
:20DA800020005356454E534B413F20202020202020200053554F4D493F2020202020202060
:20DAA000202020004E454445524C414E44533F2020202020004954414C49414E4F3F202077
:20DAC0002020202020004E4F52534B3F2020202020202020202000455350414E4F4C3F2029
:19DAE000202020202020200044414E534B3F20202020202020202020005D
:208D800056454E544F4C4120200050524F47522E205350454349414C453F0046494E4520DB
:208DA00050524F472E535045432E3F004552524F52452050524F4752414D4D4100434F444A
:208DC00049434520494E5055543A000000007300204E31202020204E32202020204E3320A5
:208DE00000492F4F20544553543F00494E47084E4720414B542E3A00555447084E4720413C
:208E00004B542E3A004552524F524520202020202020202020004E522E505247523A0000F9
:208E200000004F524520504F4D50413A000044524946545241444552494E472021212054DA
:208E4000454D502031204F46465345543A0054454D502032204F46465345543A00736563DA
:208E6000006D003F002E0050524F4752414D4D415A494F4E45202000202000DF4320004DDE
:208E8000494E0020434F4E2020002053454E5320005000200030002500680043414D4249F9
:208EA0004120434F442E3A0000000000535045474E49204D41434348494E4100005350490D
:208EC0004120434F4E54524F4C4C4F3F2000542E204420494D50554C534F3A00000000525B
:208EE000495343414C444920424F494C455220004752414E554C4920004C415641202020C6
:208F000020200053434941435155412000434F4E54494E554F203D20535441525400455296
:208F2000522E4D4F56494D204341505520200043484955444920434150552050455220007A
:208F400020202020202020202020202020202020005249454D50494D2E2041435155412025
:208F600020005249454D504945204143515541202020004F4B204C4156414747494F202097
:208F8000202020004552524F5245204C4956454C4C4F20200050524F4752414D4D41205015
:208FA000524F564120004552522E2049445241554C49434120200020202020415252455357
:208FC000544F2020202020004552522E205345435552204341504F20004552522E204C4966
:208FE000562E2053494355522E004552522E4D4F542E43455354454C4C4F004552522E2052
:209000004D4943524F20504F525441004552522E2050524F54455A2E4D4F542E00455252E0
:209020002E2053555252495343414C442E004552522E2050524553532E4143515541005308
:20904000544152543D5349202020203F3D4E4F0050524F4752414D4120424153453F202050
:209060000050524F4752414D4120424153453F3F20004E522E2050524F4752414D4D493AE8
:20908000000000204455522E4C41563A20000000000000005641522E20414C545249205631
:2090A000414C3F200054DF20534349414351554F3A000000000054DF204C41564147474991
:2090C0004F3A00000000004455522E205345504152415A3A000000004455522E5343494145
:2090E0004351554F3A000000004C49562E4C4156414747494F3A000000004C49562E2042E6
:209100004F494C45523A00000000004455522E56454E54494C2E3A00000000004252494C1E
:209120004C49414E542020000000000000414C54524920564F4C4F5249204F4B3F00464978
:209140004E452050524F4752414D4D413F2000454E474C4953483F2020202020202020000E
:20916000444555545343483F2020202020202020004652414E434149533F2020202020205A
:2091800020005356454E534B413F20202020202020200053554F4D493F20202020202020A9
:2091A000202020004E454445524C414E44533F2020202020004954414C49414E4F3F2020C0
:2091C0002020202020004E4F52534B3F2020202020202020202000455350414E4F4C3F2072
:1991E000202020202020200044414E534B3F2020202020202020202000A6
:20800000564946544520202020005350455349414C50524F472E3F20202000535045432EF3
:2080200050524F472E4B4C41523F200050524F4752414D4645494C2020202020004B4F449B
:20804000453A0000000000000000000000007300204E31202020204E32202020204E33206E
:2080600000492F4F20544553543F00494E47084E4720414B542E3A00555447084E472041C9
:208080004B542E3A004645494C484953544F52494B2020202000414E542E50524F472E3A1B
:2080A000000050554D50455449443A00000044524946545241444552494E47202121205483
:2080C000454D502031204F46465345543A0054454D502032204F46465345543A0073656B60
:2080E000006D003F002E0050524F4752414D4D4552494E4720202000202000DF4320006D7D
:20810000696E00204D4544202000205554454E200050002000300025006800454E4452453B
:20812000204B4F44453A0000000000004252595420535452304D4D454E000000004D455227
:208140004B20494E53502E3F202020202000494D50554C535449443A000000000000005622
:2081600041524D455220534B594C4C54414E4B004752414E554C4154005641534B45522061
:20818000202000534B594C4C4552202000564944455245203D2053544152542020004645A4
:2081A000494C2048455454454245562E2020004C554B4B2048455454454E20464F522000FF
:2081C000202020202020202020202020202020200056414E4E46594C4C4E494E47202020A9
:2081E000200046594C4C45522056414E4E2020202020004452494654534B4C415220202048
:20820000202020004645494C204D45442046594C4C494E47005445535450524F4752414D5B
:208220002020202020004645494C204859445241554C2E202020002020202053544F5050A1
:2082400045542020202020004645494C204B4C454D4245534B2E2020004645494C2053490D
:208260004B4B45482E4E495620004645494C204B5552564452562E202020004645494C205E
:2082800053494B4B2E425259542E20004645494C204D4F544F525645524E202000464549CF
:2082A0004C20542E4B2E53494B522E2020004645494C2056414E4E545259434B202000531D
:2082C000544152543D4A412020203F3D4E4549005354442E20564552444945523F202020FA
:2082E000005354442E20564552444945523F3F202000414E54414C4C2050524F4752414D82
:208300003A0000205641534B5449443A2000000000000000454E44524520414E4E45543F50
:208320002020202000534B594C4C4554454D503A0000000000005641534B4554454D503A8F
:2083400000000000000000534550455241534A4F4E3A000000000000534B594C4C45544978
:20836000443A000000000000004E495641205641534B3A000000000000004E495641205321
:208380004B594C4C3A00000000000056494654455449443A0000000000000000544F525287
:2083A000454D494444454C0000000000004F2E4B2E20414E4E45543F2020202020005052BC
:2083C0004F4752414D204F2E4B2E3F20202000454E474C4953483F20202020202020200029
:2083E000444555545343483F2020202020202020004652414E434149533F202020202020E8
:2084000020005356454E534B413F20202020202020200053554F4D493F2020202020202036
:20842000202020004E454445524C414E44533F2020202020004954414C49414E4F3F20204D
:208440002020202020004E4F52534B3F2020202020202020202000455350414E4F4C3F20FF
:19846000202020202020200044414E534B3F202020202020202020200033
:2084800056454E54494C4152200050524F472E2045535045432E3F2020200050524F472E2E
:2084A0002045535045432E204F4B3F004552524F522050524F4752414D41202000494E54D7
:2084C000524F20434F4449474F3A000000007300204E31202020204E32202020204E3320B9
:2084E00000492F4F20544553543F00494E47084E4720414B542E3A00555447084E47204145
:208500004B542E3A004D414E53414A4553204552524F522020004E522E505247523A0000D5
:2085200000004455522E424F4D42413A000044524946545241444552494E472021212054EC
:20854000454D502031204F46465345543A0054454D502032204F46465345543A00736563E3
:20856000006D003F002E0050524F4752414D4D4143494F4E20202000202000DF4320006D03
:20858000696E0020434F4E2020002053494E2020005000200030002500680043414D4249F1
:2085A0004520434F442E3A0000000000415041474152204D415155494E410000004D415260
:2085C00043415220494E53504543432E3F004455522E20494D50554C534F3A000000004354
:2085E000414C454E54414E444F20424F494C52004752414E554C4F20004C4156414E444F10
:2086000020200041434C415241444F2000434F4E54494E5541523D2053544152540045528E
:20862000522E4D4F56494D204341504F544100434552524152204341504F54412020200063
:20864000202020202020202020202020202020200050415241204C4C454E4152204147551B
:208660004100434F4749454E444F2041475541202020005055454445204C4156415220208A
:20868000202020004552524F52204C4C454E41444F2020200050524F4752414D412044456F
:2086A0002054455354004552522E204859445241554C49434120002020494E5445525550B6
:2086C00043494F4E202020004552522E5345435552204341504F5441004552522E4E49569C
:2086E000454C2053454755522E004552522E4D4F562E43414E4153544120004552522E5359
:20870000454E532E20505545525441004552522E204D4F544F522D50524F542E0045525203
:208720002E50524F5445432E5445524D2E004552522E50524553494F4E20414755410053E2
:20874000544152543D53492020203F3D4E4F4E00204441544F5320464142524943413F203C
:2087600000204441544F5320464142524943413F3F004E522E2050524F4752414D413A0057
:20878000000000204455522E4C41563A20000000000000002043414D422E4F54524F53204B
:2087A00056414C3F0054DF2041434C415241444F3A000000000054DF204C415641444F3A8F
:2087C0000000000000000053455041524143494F4E3A0000000000004455522E41434C4150
:2087E0005241444F3A000000004E49562E2054414E5155453A00000000004E49562E204259
:208800004F494C45523A00000000004455522E56454E54494C2E3A000000000050524F441B
:208820002E204252494C4C4F0000000000204F54524F2056414C2E204F4B3F2020002046F2
:20884000494E414C2050524F4752414D413F00454E474C4953483F202020202020202000F3
:20886000444555545343483F2020202020202020004652414E434149533F20202020202063
:2088800020005356454E534B413F20202020202020200053554F4D493F20202020202020B2
:2088A000202020004E454445524C414E44533F2020202020004954414C49414E4F3F2020C9
:2088C0002020202020004E4F52534B3F2020202020202020202000455350414E4F4C3F207B
:1988E000202020202020200044414E534B3F2020202020202020202000AF
:2089000056454E54494C415420005350454349414C50524F472E3F20202000535045432E71
:2089200050524F47204B4C41523F200050524F4752414D46454A4C2020202020004B4F449F
:20894000453A0000000000000000000000007300204E31202020204E32202020204E332065
:2089600000492F4F20544553543F00494E47084E4720414B542E3A00555447084E472041C0
:208980004B542E3A0046454A4C484953544F52494B3F20202000414E542E50524F472E3AF2
:2089A000000050554D50455449443A00000044524946545241444552494E4720212120547A
:2089C000454D502031204F46465345543A0054454D502032204F46465345543A0073656B57
:2089E000006D003F002E0050524F4752414D4D4552494E4720202000202000DF4320006D74
:208A0000696E00204D4544202000205544454E20005000200030002500680041454E445246
:208A200045204B4F44453A0000000000534C554B20535452304D4D454E000000004D4152DF
:208A40004B455220494E53502E3F20202000494D50554C535449443A0000000000000056C2
:208A600041524D455220534B594C4C54414E4B004752414E554C4154005641534B45522058
:208A8000202000534B594C4C4552202000564944455245203D20535441525420200046459B
:208AA0004A4C204841455454454245562E20004C554B4B204845415454454E20464F5200B3
:208AC000202020202020202020202020202020200056414E44500846594C444E494E47209A
:208AE0002000500846594C4445522056414E4E2020200044524946544B4C41522020202062
:208B00002020200046454A4C204D2E2046594C444E494E47005445535450524F4752414D66
:208B200020202020200046454A4C204859445241554C494B2020002020202053544F505051
:208B4000455420202020200046454A4C204B4C454D4245534B2E20200046454A4C20534902
:208B60004B4B4552482E4E49560046454A4C204B555256454452455620200046454A4C20E5
:208B80004430524B4F4E54414B54200046454A4C204D4F544F52564145524E200046454A90
:208BA0004C20542E4B2E53494B522E20200046454A4C2056414E445452594B202020005340
:208BC000544152543D4A412020203F3D4E454A005354442E20564552444945523F202020F0
:208BE000005354442E20564552444945523F3F202000414E54414C2050524F4752414D3A8B
:208C0000000000205641534B4554443A200000000000000041454E44524520305652494791
:208C2000413F202000534B594C4C4554454D503A0000000000005641534B4554454D503A46
:208C40000000000000000053455041524154494F4E3A000000000000534B594C4C45544973
:208C6000443A000000000000004E4956454155205641534B3A00000000004E495645415557
:208C800020534B594C3A000000000056454E54494C2E5449443A00000000000054305252F4
:208CA000454D494444454C0000000000004B4C4152203056524947453F2020202000505268
:208CC0004F4752414D204F2E4B2E3F20202000454E474C4953483F20202020202020200020
:208CE000444555545343483F2020202020202020004652414E434149533F202020202020DF
:208D000020005356454E534B413F20202020202020200053554F4D493F202020202020202D
:208D2000202020004E454445524C414E44533F2020202020004954414C49414E4F3F202044
:208D40002020202020004E4F52534B3F2020202020202020202000455350414E4F4C3F20F6
:198D6000202020202020200044414E534B3F20202020202020202020002A
:20FF000001010A141E28323C46505152535455565758595A0001010A141E28323C3D3E3F92
:20FF200040414243444546000A141E28323C000A0F14191E23282D32373C0000010F14195C
:18FF40001E23282D3C4B5AFF000000010300010600000300000000FF26
:20FD0000DD8DDF8F18DF91135002107F005CBDEC772608BDEC7D26031550021350400B7C05
:20FD2000007A967A810F2E0D20177A007A967A81002702200C135040051550402003145089
:20FD4000401350010EBDEBF47C008C968C81072E07200B7F008C2006BDEC70155001134F31
:20FD600020037C005D134F40037C005E134F10037C005C7C0063860A91632E33134D800512
:20FD8000DE5708DF577C0079144E107C00597C005B7C00667C0067134F8007DC5FC3000130
:20FDA000DD5F7C005A7F0063134F02037C0078966427087A00642603154E04966527087AB9
:14FDC00000652603154E088640B71025DC8DDE8F18DE913BEC
:20E000008600B710248693B710397F10358683B71026863EB710098E00FF8600B760018677
:20E02000FFB760008604B760018600B7600386E0B760028604B76003BD940018CE01F4BD7C
:20E0400093AEBDF7A2861497DF860097287F00327F00457F0046BDF894BDF256BDF7A2BD39
:20E06000F952BDEAD3BDEAA5BDEE27B6103181FF27037EE088BDEE59B6103281FF27037E12
:20E08000E088BDF7A27EA144860097289728BD9309BDEC8F2700BDEC7D2706154E407EA08F
:20E0A000007EE2CE154E41BD9309CCC096BD9343DC3FBD92F1BD931FCCC0A2BD9343DC41D8
:20E0C000BD92F1CCC119BD9343BD969D124C01F9124C04F5BD9309B6B715978BB6B7149713
:20E0E0008A972CCCC0BFBDF107978ACEB714BD966A968B972CCCC0CEBDF107978BCEB715AD
:20E10000BD966A18CE01F4BD93AEBD9309BD931FCCC050BD9343BD930086019723BDED07F0
:20E12000962BBD92D1CCC113BD9343BD930086079723BDED3F962BBD92D1CCC113BD934337
:20E14000BD9300860D9723BDED77962BBD92D1CCC113BD9343BDE709965127037EE653BDBB
:20E16000EC7D262220B0BD9309CCC061BD9343BD931FCCC2BFBD9343BD969D124C0107128E
:20E180004C04037EE266145001BD9300CCC085BD9343BD931FCCC2BFBD9343BD969D124C70
:20E1A00001E1124C04DDBD9300CCC1C0BD9343BD9300CEB7E0A600BD92D1CCC0E5BD93438F
:20E1C000CEB7E0A601BD92D1CCC0E5BD9343CEB7E0A602BD92D1CCC0E5BD9343CEB7E0A6D3
:20E1E00003BD92D1CCC0E5BD9343CEB7E0A604BD92D1BD969DBD9300CCC1C0BD9343BD9359
:20E2000000CEB7E0A605BD92D1CCC0E5BD9343CEB7E0A606BD92D1CCC0E5BD9343CEB7E030
:20E22000A607BD92D1CCC0E5BD9343CEB7E0A608BD92D1CCC0E5BD9343CEB7E0A609BD9273
:20E24000D1BD969DBD9300CCC1C0BD9343BD9300CCC13DBD9343BD969D124C0109124C0466
:20E26000058663BDF349BD9309CCC215BD9343BD931FCCC2BFBD9343BD969D124C01081270
:20E280004C040486019728BD9300CCC1C0BD9343BD9300CCC14EBD93439627BD92D1BD96C6
:20E2A0009D124C020F7C0027861591272ED98601972720D3BD9300CCC01BBD9343BD969DA3
:20E2C000124C0107124C04037EF5377EE0A4BDF952144E40BDF7A2BD9309963397529634F2
:20E2E0009753154E03154E01BDE9D7965127037EE653BDED072646154E30BD9300CCC1AFE9
:20E30000BD9343BD931FCCC1D1BD9343BD969D124C01F9BDEA3E8602915127D6860191510D
:20E3200027C3144E30BD9309BD931FCCC1E2BD9343144E32BDE9138601915127A8144E03AD
:20E3400086019745144E30BD931FCCC1F3BD9343BD969D124C01F9124C040D7EE387BDE901
:20E36000D7965127227EE6E1BDEC95260DBDEA3E965127037EE6537EE347BDE9D796512700
:20E38000037EE6537EE347155080144E30BD931FCCC1C0BD9343BD931FCCC111BD9343961F
:20E3A000458100272D9645BD92D1CCC113BD9343BDE695967BBD92D1CCC0FFBD9343CCC101
:20E3C00013BD934396548100270BCCC170BD93432003BD931FBD969D124C0413124C022EE5
:20E3E0007C0045963591452C9E860197452098BDEC95260DBDEA3E965127037EE6537EE357
:20E4000087BDE9D7965127037EE6537EE3874F91452600BD931FCCC1C0BD9343144E301408
:20E420005080BDE695BDEBED7F00577F0058144D80BDE709965127037EE653CC00091A93BA
:20E44000572EEEBDEA3E965127037EE65318CE07D0BD93BFBDE913965127037EE387CC0052
:20E460000BDD57BDEBCE18CE01F4BD93AEBDEBDF18CE01F4BD93AEBDEBB69627C60A3D186E
:20E480008FBD93AEBDE709965127037EE653BDEFFDCC000E1A93572EEBBDEC1EBDE70996D0
:20E4A0005127037EE653BDEFFDCC00171A93572EEBBDEBB618CE0064BD93AECCC179DD7C7C
:20E4C000144E80BDE709965127037EE65318CE0190BD93AEBDEC40BDEFFDCC001B1A9357F3
:20E4E0002EE14F91542703BDEBD8BDE709965127037EE653BDEFFDCC001BD3551A93572ED0
:20E50000E9BDEC54BDE709965127037EE653BDEFFDCC001BD355D3881A93572EE7154D8092
:20E52000BDEC1E18CE01F4BD93AEBDEC5BBDEDEB2615BD931FCCC1C0BD9343154E80BD93E5
:20E540001FCCC15FBD9343BDE709965127037EE6537A00537A0053BDEDEB270220087C00AC
:20E56000537C005320E17C00537C0053BDEBE618CE01F4BD93AEBDEBCE144D80CCC183DD2F
:20E580007C144E80BDE709965127037EE653DC86C3001BD355D3881A93572EE8BDEC4018CA
:20E5A000CE01F4BD93AEBDEC6218CE01F4BD93AEBDEC69DC391A8300002725CCC000DD7CC1
:20E5C000BDEBC7BDE709965127037EE653DC86C30028D355D388D3391A93572EE6BDEC3981
:20E5E000962881012724154D80154E80BD931FCCC1C0BD93437F00577F0058144E301550D8
:20E6000080BDF08ABDE9D77EE387BDF08ABD931FCCC1C0BD9343154E80BDE9D7BD9309158A
:20E620004EB0CCC179DD7CCCC215BD9343144D807F00577F0058BDE709965127037EE65344
:20E64000BDEC7D2608CC02321A93572EE9BD93097EE4138601915126037EE2E5860291513C
:20E6600026037EE2F28607915126037EE387860A915126037EE2CE860B915126037EF39138
:20E68000860C915126037EE0A4860D915126037EF13E7EEB879645C6033DC300A38FA60024
:20E6A000975408A600977B972BC6B73DDD559637C6033DDD88D355DD7E9636C6033DDD8611
:20E6C000D37EDD7E9638498102270BC6033DDD39D37EDD7E2005CC000020F3C30028DD7EB0
:20E6E00039BD9300BD931FCCC237BD934318CE01F4BD93AEBD931FCCC1C0BD934318CE01BB
:20E70000F4BD93AEBDEAA520D8BDEF53134E2007134E1003BDEEBCBD92AA134E0126BDED36
:20E7200077261E860F91662E1BBD9300154E30CCC259BD93438605BDF349154E01BDE6E180
:20E74000397F0066BDEC952743BDEC7D2745124F0148144F10860A915C2E4CBDEAD3BDEA2C
:20E76000A5144F01BDEAA5154E80BDEC952603154E0C144E30BD9309BDE9D7154F01134E5D
:20E78000010586079751398601975139BDECCB270920B6BDEC77270920B4BDED012702208B
:20E7A000A8154F107F005CBDED012720BDECB9271B144F208600915D2E18BD931FCCC26A28
:20E7C000BD93438606BDF349BDEAF839154F207F005D7A0052BDED772718BDEDAF26137CAF
:20E7E00000527A00527A0052BDEDAF260DBDEB9320087C0052BDEBFB20067C00527C00520D
:20E800007A0053BDED3F2722BDEDEB261D7C00537A00537A0053BDEDEB2617BDECE3261222
:20E82000BDECFB260DBDEB9A20087C0053BDEC0220067C00537C0053BDEC95271DBDECD15D
:20E840002718144F40865B915E2E15CCC27BBD93438607BDF349BDEA2539154F407F005E1B
:20E86000BDECE92720BDECA3271B124F0817144F08BD9309CCC28CDD6DBD93438608BDF3B8
:20E8800049BDEB1D39BDEC9B271B124F0417144F04BD9309CCC29DDD6DBD93438609BDF328
:20E8A00049BDEB1D39134E0217BDECFB2612BDED3F260D144F80CC044C1A935F2E11201A1B
:20E8C000154F807F005F124F0227BDEC17202DBDEBAF7F0078144F022022BDEC17BD9309D1
:20E8E000CCC2AEDD6DBD9343860ABDF349BDEB1D39860691782E05154F0220CEBDECCB27C1
:20E900000B863D915A2E0BBDEC0920067F005A7F0051397F0061BDE7099651270139BDEDCC
:20E92000772709BDED0727047F005139BDEDAF261B7A00537A0053BDEDEB27087C00537C08
:20E94000005320087C00537C005320CABDED3F27C5BDE7099651270139124F02F47F005BB9
:20E9600018CE03E8BD93AEBDEBCE963B2703BDEBE6BDE7099651270139965B815B2E1BBD01
:20E98000ED0727ED7F0079BDE7099651270139BDED0727DD861991792EEDBDEC40BDEC6215
:20E9A000BD931FCCC1E2BD93437C0061860A91612E22BDED77270B861991612E17BDED075D
:20E9C0002612BD9300CCC204BD93438602BDF349BDEB34397EE916134E2007134E1003BDBE
:20E9E000EEBCBDE7099651270139124E04E9124E08E57F0059BDE70996517F005127013941
:20EA0000BDECAB2607BDEC107F005139BDEC09BDEBA8860691592EDDBDECB12711863D914A
:20EA2000592ED22009BDEAA5BDEAD37EE6E1BD9300CCC226BD93438603BDF34920E7BDEC80
:20EA4000952617BDEBA118CE01F4BD93AEBDE7099651270139BDEC95271D18CE07D0BD933E
:20EA6000AE7F005139BDE7099651270139862F915A2EF27F005139BDECB12617864E915ACB
:20EA80002ECBBD9309CCC19EBD93438601BDF3497EEA25BD931FCCC248BD93438604BDF347
:20EAA00049BDEB5C39BDEC17BDEC54BDEC1EBDEC40BDEBFBBDEC02BDEC10BDEC09BDEC6998
:20EAC000BDEC39BDEC5BBDEC62BDEC32BDEC70154E80397F00577F00587F005F7F00607F4C
:20EAE00000617F00627F005D7F005F7F004C154D80154E3C154FF039BDEAD3BDEAA5BDE9D5
:20EB0000D7BD969D124C01F9124C04F5BD9309124E010586029751398607975139BDEAD3EF
:20EB2000BDEAA5BDE9D7154E03BD9300DC6DBD93437EE6E1BDEAD3BDEAA5BDE9D7154E335C
:20EB4000BD931FCCC18DBD9343BD969D124C01F9124C04F5BD93098601975139BDEAD3146B
:20EB60004F01BDEAA5154F01BDE9D7BD969D124C01F9124C04F5BD9309124E01058602979A
:20EB800051398607975139BD9300CCC02CBD93437EE6E1CE60001C000839CE60001C000484
:20EBA00039CE60001C000239CE60001C000139CE10081C000239CE10081C0004144E043931
:20EBC000CE10081C001039CE10081C000839CE10081C0020144E0839CE10001C008039CE61
:20EBE00010001C004039CE10001C002039CE10001C001039CE10001C000839CE60001D0054
:20EC00000839CE60001D000439CE60001D000239CE60001D000139CE10081D000239CE1004
:20EC2000081D0004124F0109865B97659764144E0439CE10081D001039CE10081D00083939
:20EC4000CE10081D0020124F0109865B97659764144E0839CE10001D008039CE10001D00FC
:20EC60004039CE10001D002039CE10001D001039CE10001D000839B66002841039B660024A
:20EC8000840839B66002840439B66002840239B66002840139B6100A848039B6100A844088
:20ECA000884039B6100A8420882039B61000840439B610008402880239B61000840139B62E
:20ECC0006000840839B66000840439B66000840239B66000840139B61000844039B6100006
:20ECE000842039B61008840239B61008840439B61008841039B61008840839B6100884207B
:20ED000039B610008410398603B7103018CE0001BD93AECE10301E00800586019748397FF3
:20ED20000048F6103486C43DCE0032028FCE000A028F17972B913D2E0386003986013986F3
:20ED400002B7103018CE0001BD93AECE10301E00800586019748397F0048F6103386C43DFE
:20ED6000CE0032028FCE000A028F17972B913E2E038600398601398604B7103018CE0001D9
:20ED8000BD93AECE10301E00800586019748397F0048F6103186C43DCE0032028FCE000A37
:20EDA000028F17972B913D2E038600398601398600B7103018CE0001BD93AECE10301E00DD
:20EDC000800586019748397F0048F61031C02C86413DCE0095028FCE0001028F17800A9B91
:20EDE0008A91522E038600398601398601B7103018CE0001BD93AECE10301E00800586015B
:20EE00009748397F0048F61032C02C86413DCE0095028FCE0001028F17800A9B8B91532EBE
:20EE2000038600398601398600B7103018CE0001BD93AECE10301E00800586019748397F1F
:20EE40000048F61031C02C86413DCE0095028FCE0001028FC00ADB8A398601B7103018CE23
:20EE60000001BD93AECE10301E00800586019748397F0048F61032C02C86413DCE009502EF
:20EE80008FCE0001028FC00ADB8B3997977F0096BD95BE8620BD960FCE009CA600812027E7
:20EEA00004BD952A390820F3DD96BD95BE8620BD960FCE009C20E4BD952A3939134E20FB1B
:20EEC000BDECBF270413504019BD9300BD930086019723BDEE2717BD92D1CCC0FBBD9343DF
:20EEE0002016BD9300BD930086019723CCC0F8BD9343CCC0F8BD9343BDECC5270413504091
:20EF000016BD9300860B9723BDEE5917BD92D1CCC0FBBD93432013BD9300860B9723CCC091
:20EF2000F8BD9343CCC0F8BD934313508016BD930086079723CCC111BD93439645BD92D173
:20EF4000154E1039BD930086079723CCC0F8BD934320ED134E8056BD931FDC7CBD9343DCDD
:20EF60007E93570C59490C59490C59490C59490C5949CE0064028FDD80CE003C028FD782AF
:20EF8000863C3DDD83DC809383D7859682BD92D1CCC0E1BD9343968581092E06CCC115BDD4
:20EFA00093439685BD92D1CCC0DDBD9343398FBD952A393C183C3637BD931FCCC117BD9367
:20EFC00043200CC61086104A26FD5A26F82005BDEC7D27FB3332183838393C183C3736BD24
:20EFE0009309CCC117BD93433233183838393C183C3736BDEC7D27FB323318383839BD935D
:20F0000000BD931F9657BD92F1398600CEB709BD966A8600CEB70908BD966A8600CEB71155
:20F02000BD966A8600CEB71108BD966A8600CEB713BD966A8600CEB716BD966A8600BDF343
:20F04000498600BDF3498600BDF3498600BDF3498600BDF3498600BDF3498600BDF34986E7
:20F0600000BDF3498600BDF3498600BDF3498603CEB721BD966A8608CEB722BD966ABD936B
:20F0800009CCC0AEBD93437EF087B6B7169744FCB709DD3FFCB711DD41B6B71397439B7B1D
:20F0A000813B2E569743DC3FC30001DD3F96449B37813B2E02200C803C974496438B0197E4
:20F0C00043964497449643CEB713BD966A9644CEB716BD966ADC41CEB711BD966ADC411734
:20F0E000CEB71108BD966ADC3FCEB709BD966ADC3F17CEB70908BD966A39803C9743DC41DE
:20F10000C30001DD41209FDD6DBD9300DC6DBD9343962C81092E06CCC113BD9343962CBDA6
:20F1200092D1BD969D124C0212962C8B01972C81142E0220D48601972C20CE962C39154EAA
:20F1400040BDF952BD9300BD931FCCC0F8BD9343BDEC772708CCC0E5BD93432003BDF24C20
:20F16000BDEC7D2708CCC0E5BD93432003BDF24CBDEC832708CCC0E5BD93432003BDF24C9B
:20F18000BDEC892708CCC0E5BD93432003BDF24CBDEC8F2708CCC0E5BD93432003BDF24C63
:20F1A000BDEC952708CCC0E5BD93432003BDF24CBDEC9B2708CCC0E5BD93432003BDF24C2B
:20F1C000BDECA32708CCC0E5BD93432003BDF24CBDECAB2708CCC0E5BD93432003BDF24CED
:20F1E000BDECB12708CCC0E5BD93432003BDF24CBDECB92708CCC0E5BD93432003BDF24CB1
:20F200008681BD9510BDED07962BBD92D1CCC113BD93438687BD9510BDED3F962BBD92D187
:20F22000CCC113BD9343868DBD9510BDED77962BBD92D1CCC113BD9343BDEC7D26037EF133
:20F2400044BDEC7D26FBBD93097EF241CCC115BD9343397EF30D963C97298609972ABDF39B
:20F260003B26F0963597298609972ABDF33B26E396349729865A972ABDF33B26D6963397FC
:20F28000298646972ABDF33B26C996379729863C972ABDF33B267696379729863C972ABD7A
:20F2A000F33B266996369729863C972ABDF33B265C963D9729865A972ABDF33B264F963EAD
:20F2C0009729865A972ABDF33B264296389729865A972ABDF33B2635963B97298601972A2C
:20F2E000BDF33B2628968A97298614972ABDF33B261B968B97298614972ABDF33B260E967D
:20F300002797298615972ABDF33B260139BDF906860A978A978BBDF811968ACEB714BD96FE
:20F320006A968BCEB715BD966A8603973CCEB706BD966A8662BDF3497EE6E19629912A2285
:20F34000022003860139860039CEB7E0E600BD966A0817E600BD966A0817E600BD966A0875
:20F3600017E600BD966A0817E600BD966A0817E600BD966A0817E600BD966A0817E600BDCB
:20F38000966A0817E600BD966A0817E600BD966A39BD931FCCC2BFBD9343BDF952154E02F4
:20F3A0007F0032BD9300BDF63DBD969D124C0208BDF64CBDF7A220D9BDF7A2BD931FCCC263
:20F3C000BFBD9343BD9300CCC2D0BD9343BD969D124C011E124C041ABD9300CCC2E1BD93A2
:20F3E00043BD969D124C010A124C0406BDF9067EF54E7C0032BD9300CCC1C0BD9343BD935E
:20F4000000CCC2E1DD6BBDF56ABD969D124C0205BDF64C20E086019745BD9300CCC111BDB7
:20F4200093439645BD92D18603D6453DC300A3C30000DD2E8FA60081FF26048600A7008159
:20F44000002708CCC103BD93432006CCC10ABD9343CCC170BD9343BD969D124C0210DE2E0E
:20F460006C008602A10026026F00DF2E20ABBD9300CCC111BD93439645BD92D1CCC303BDBD
:20F4800093438603D6453DC300A3C30001DD2E8FA60081FF26048601A700BD92D1CCC0FFC8
:20F4A000BD9343BD969D124C0210DE2E6C008609A1002ABA8601A70020B47C004596358BB4
:20F4C00001914527037EF4197C0032BD9309BD931FCCC2BFBD9343BD9300CCC314BD9343C4
:20F4E000BD969D124C0167124C0463BD9300CCC1C0BD9343BD9300CCC303DD6BBDF56ABD5E
:20F50000969D124C0205BDF64C20E97C0032860991322AD77F0032BD9300CCC00ABD934320
:20F52000BD931FCCC2BFBD9343BD969D124C0107124C04037EE0A4BD9300CCC3ADBD9343A0
:20F54000BD969D124C0207860297327EF4F4BD9300CCC3BEBD9343BD969D124C02037EF3A9
:20F5600091BDF811BD93097EE2CEBD931FCCC2BFBD9343BD93008611D6323DD36BBD934361
:20F580008601913226059635BD92D186029132260B9634BD92D1CCC0FBBD9343860391323F
:20F5A000260B9633BD92D1CCC0FBBD934386049132260B9637BD92D1CCC04EBD93438605B4
:20F5C0009132260B9636BD92D1CCC04EBD9343860691322611963DBD92D1CCC117BD93432E
:20F5E000CCC0F8BD9343860791322611963EBD92D1CCC117BD9343CCC0F8BD93438608910C
:20F6000032262196384981022712BD92D1CCC04EBD9343CCC0F8BD93437EF624CCC115BD03
:20F62000934320E9860991322612963B2708CCC103BD93432006CCC10ABD934339BD930065
:20F640008611D63C3DC3C3CFBD9343398600913226127C003CBDF7A28609913C2A6F7F00A0
:20F660003C7EF79E8601913226107C0035860991352A5A860197357EF79E86029132262337
:20F680007F0068CCFF008FD6683AA600810026067F00687F003491342E057C006820E4974D
:20F6A00034202A8603913226277F0068CCFF158FD6683AA600810026067F00687F003391E8
:20F6C000332E057C006820E497337EF79E7EF79E8604913226247F0068CCFF288FD6683A74
:20F6E000A600810026067F00377F006891372E057C006820E497377EF79E860591322623BF
:20F700007F0068CCFF2F8FD6683AA600810026067F00687F003691362E057C006820E49799
:20F7200036207B860691322612963D8B0A973D8663913D2A697F003D7EF79E8607913226A6
:20F7400012963E8B0A973E8663913E2A517F003E7EF79E8608913226237F0068CCFF3B8F40
:20F76000D6683AA60081FF26067F00687F003891382E057C006820E49738202286099132DA
:20F78000260F963B27057F003B20138601973B200DCCC02CBD934318CE03E8BD93AEBDF9F4
:20F7A0004839963C81002607CCC480DD69202181012607CCC900DD69201681022607CCCDA8
:20F7C00080DD69200B81032607CCC000DD69204081042607CCD200DD69203581052607CCEB
:20F7E000D680DD69202A81062607CC8D80DD69201F81072607CC8000DD69201481082607E0
:20F80000CC8480DD69200981092605CC8900DD69399627CEB6D0BD966A9633CEB700BD96B1
:20F820006A9634CEB701BD966A9635CEB702BD966A9636CEB703BD966A9637CEB705BD9687
:20F840006A963CCEB706BD966A963DCEB707BD966A963ECEB717BD966A9638CEB719BD961C
:20F860006A963BCEB720BD966A963FCEB709BD966A9641CEB711BD966ABDF948C600CEB659
:20F880000018CE00A318A600BD966A0818085CD14726F239B6B7009733B6B7019734B6B79A
:20F8A000029735B6B7039736B6B7059737B6B706973CB6B707973DB6B717973EB6B71997F9
:20F8C00038B6B720973BFCB709DD3FFCB711DD41B6B7139743B6B714978AB6B715978BB681
:20F8E000B7169744B6B6D09727BDF256BDF948C600CEB60018CE00A3A60018A70008180803
:20F900005CD14726F33986059727863C9733865597348603973586149736861E97378628CA
:20F92000973D860A973E860197388600973BBDF948C600CEFF4818CE00A3A60018A7000811
:20F9400018085CD14726F3398603D6353DCB03D7473918CE012CBD93AE7F005018CE1024D1
:1AF96000181C0040BDEAD3154FFF154E801450408600977A0E18CE00C83929
:209200009626810F2E0786809B267E921186B09B26BD95108600B76001860FB760008604B8
:20922000B7600118CE6002181C0020181C0040181C0080B6600084F0972418CE6002181D90
:209240000080181C0080B6600084F09725181D00E08600B7600186FFB760008604B76001A3
:20926000962546464646840F9A24972439A600271A3696228101260732BD93757E92833296
:20928000BD93920886194A26FD20E2399626810F2E0ACC0000DB26188F7E92A6CC0011DB37
:2092A00026830010188F18A60039BD9200BD928C9124260F96264C9726811F2E01398600F0
:2092C000972639BD9400BD94CCBD9328860097263997977F0096BD95BE8620BD960FCE000D
:2092E0009CA60081202707BD926DBD9328390820F0DD96BD95BE8620BD960FCE009C20E1E2
:20930000860197228600972339BD9300CCC1C0BD9343BD931FCCC1C0BD9343BD9300398606
:209320000297228600972339BD932FBD933939BD94F4CC0000BDEFAE39BD94EECC0011BD3B
:20934000EFAE3983C000D3698FA600810027183C3696228101260732BD93757E936232BD91
:20936000939238087E9349962281012604BD932F39BD93393918CE0000D623C100270BC1BD
:20938000112E0E18085AC10026F918A7007C0023393918CE0011D623C100270BC1112EF182
:2093A00018085AC10026F918A7007C002339183C3CCE01470926FD38180926F418383918D6
:2093C0003C3CCE01470926FD38180926F418383936B66000840F972D3284F09A2DB76000B0
:2093E0003918CE6002181D0040BD93D018CE6002181C0080181D0080181C0040BD953A396D
:2094000018CE6002BD953ABD953A18CE6002181D00A0181C00408630BD93E18630BD93E18D
:209420008630BD93E18620BD93E18628BD949EBD953A8606BD949EBD953A8614BD949EBDF8
:20944000953A860CBD949EBD953A8601BD949EBD953A18CE6002181C002018CE6002181D15
:209460000020181D00408640BD949EBD953A18CE6002181C0020CE957EDF6D8640972BDEE7
:209480006DA60008DF6DBD949EBD953A962B4A972B810026EA18CE6002181C00203918CED1
:2094A0006002973184F0BD93D0BD94BB9631840F48484848BD93D0BD94BB39181D00401876
:2094C0001C0080181D0080181C00403918CE6002181D00208601BD949EBD953ABD953A184B
:2094E000CE6002181C0020398680BD95103986C0BD95103918CE6002181D00208602BD94B7
:209500009EBD953ABD953A18CE6002181C00203918CE6002181D0020BD949EBD953ABD9556
:209520003A18CE6002181C002039A600270BBD949E0886194A26FD20F13918CE0014BD93AD
:20954000AE3936375F8164251A5C8064816424F9CB303617BD949E325F810026068630BD0A
:20956000949E4F810A250F5C800A810A24F9CB303617BD949E328B30BD949E333239040068
:209580000E111F1111000A000E111F1111000A000E1111110E0003041F101E101F0002051E
:2095A0001F101E101F0003041F111F1111001100111111111F000E11101010150E037F004F
:2095C000937F00947F009586109799CE009586039798A600979A840F80052B06969A8B0312
:2095E000979A969A84F080502B06969A8B30979A969AA700097A009826D87800977900966B
:209600007900957900947900937A009926BD39CE009CA700088C00A026F8CE000096938416
:209620000F27058B30979C089694444444442606D69CC12027058B30979D089694840F263A
:2096400006D69DC12027058B30979E089695444444442606D69EC12027048B30979F969589
:20966000840F8B3097A07F00A13937183CC616F7103BE700C617F7103B18CE000ABD93AE6F
:209680007F103BC602F7103BA700C603F7103B18CE000ABD93AE7F103B1838333936373C27
:2096A000183C154C07BDEC7726FBBDEC7D26F6BDEC8326F118CE0019BD93AEBDEC7726E500
:2096C000BDEC7D26E0BDEC8326DB134E400ABDE709965127037EE653BD92AABD973BBDECE0
:2096E0007727037E970ABDEC7D27037E96F6BDEC8327D77E971E18CE0019BD93AEBDEC7DD0
:2097000027C8144C02145002202818CE0019BD93AEBDEC7727B4144C01145002201418CE71
:209720000019BD93AEBDEC8327A0144C041450022000145001183838333239134E2007130F
:079740004E1003BDEEBC3921
:20A00000BDA10DBD930986009730BD9300CCC03DBD93439630BD92D1BD931FCCC2BFBD9391
:20A0200043BD969D124C0107124C04037EA0427C00309630810A27037EA00A860097307EA8
:20A04000A00ACC0000DD2EBD9300CCC03DBD93439630BD92D1DC2EBD92F1BD931FCCC2BFE7
:20A06000BD9343BD969D124C0107124C04037EA089DC2EC30001DD2E1A83000A27037EA023
:20A0800047CC0000DD2E7EA0479630B1B7212617962FB1B72226102007860C97517EE653D4
:20A0A000860B97517EE653BD930996308107260ADC2E1A83000226022007860A97517EE6C5
:20A0C0005386009730BD9300CCC03DBD93439630BD92D1BD931FCCC2BFBD9343BD969D12FD
:20A0E0004C0107124C04037EA0FD7C00309630810A27037EA0C5860097307EA0C59630810B
:20A100000926B7BD9309860D97517EE653BDEC7D26FBBD9300CCC0E7BD9343BD931FCCC234
:20A12000BFBD9343CC0000DD57144D80DC571A83000A2E05BDEC7727037EA0BABDEC7D2770
:20A14000EB7EA003BDF952BDF7A286009728154E40BD9309CCC11BBD9343B6B721BD92D16B
:20A16000B6B722BD92D1BD931FCCC2BFBD9343BD969D124C0107124C04037EA1807EA21651
:20A18000BD930986009730BD9300CCC03DBD93439630BD92D1BD931FCCC2BFBD9343BD96E5
:20A1A0009D124C0107124C04037EA1BF7C00309630810A27037EA187860097307EA187CCCD
:20A1C0000000DD2EBD9300CCC03DBD93439630BD92D1DC2EBD92F1BD931FCCC2BFBD934349
:20A1E000BD969D124C0107124C04037EA206DC2EC30001DD2E1A83000A27037EA1C4CC0025
:20A2000000DD2E7EA1C49630CEB721BD966A962FCEB722BD966ABD9309CCC12CBD93437EDB
:02A22000A21F7B
:008000017F
